:020000040000FA
:020000002C28AA
:080008000528A000030E83018E
:10001000A10083120C1C0E280C101010210E83005E
:10002000A00E200E090026201F201F201F201F20A9
:100030001F201F201F201F20A30D03110800A30D48
:10004000A20D031C2628A20203140800A202031812
:100050000800A207031008008312870185010730FA
:10006000990093014C30950081309F0083160D302C
:1000700085008701013091003F30920020309F00C1
:10008000CF308100831212158B178312640005197B
:100090004728051D49288F018E01101405194E2887
:1000A000101020308E024E308F020F08273C031DA7
:1000B000031C5B286128951310308E0227308F02B5
:1000C00069289517FF308F068E06EF308E02D830E4
:1000D0008F020F08A2000E08A3002830132003107F
:1000E00023080339A400A40DA40DA40DA40D150824
:1000F000CF39240495002308FC39A400A40CA40CD7
:06010000240893004528CD
:00000001FF
